 BUSPCIE950

 Timestamp is 49d37576 (Wed Apr 01 15:08:54 2009)

 Preferred load address is 10000000

 Start         Length     Name                   Class
 0001:00000000 000009ceH .rdata                  CODE
 0001:000009d0 00000027H .rdata$debug            CODE
 0001:000009f8 000023dcH .text                   CODE
 0001:00002dd4 0000000cH .xdata                  CODE
 0001:00002de0 00000028H .idata$2                CODE
 0001:00002e08 00000014H .idata$3                CODE
 0001:00002e1c 000000a8H .idata$4                CODE
 0001:00002ec4 00000016H .idata$6                CODE
 0001:00002ee0 00000057H .edata                  CODE
 0002:00000000 000000a8H .idata$5                DATA
 0002:000000a8 0000044cH .data                   DATA
 0002:000004f8 0000010cH .bss                    DATA
 0003:00000000 00000088H .pdata                  DATA

  Address         Publics by Value              Rva+Base       Lib:Object

 0000:00000000       ___safe_se_handler_table   00000000     <absolute>
 0000:00000000       ___safe_se_handler_count   00000000     <absolute>
 0001:0000001c       ??_C@_1BI@IGMEDLLH@?$AA?$CF?$AAs?$AA?2?$AAU?$AAn?$AAi?$AAm?$AAo?$AAd?$AAe?$AAm?$AA?$AA@ 1000101c     buspcie950.obj
 0001:00000034       ??_C@_1BK@BFIEKNFP@?$AAF?$AAr?$AAi?$AAe?$AAn?$AAd?$AAl?$AAy?$AAN?$AAa?$AAm?$AAe?$AA?$AA@ 10001034     buspcie950.obj
 0001:00000050       ??_C@_19OBNDINH@?$AAP?$AAo?$AAr?$AAt?$AA?$AA@ 10001050     buspcie950.obj
 0001:0000005c       ??_C@_1BG@KCOOGCNN@?$AAD?$AAe?$AAv?$AAi?$AAc?$AAe?$AAT?$AAy?$AAp?$AAe?$AA?$AA@ 1000105c     buspcie950.obj
 0001:00000074       ??_C@_1BK@HFHDBJKI@?$AAU?$AAn?$AAi?$AAm?$AAo?$AAd?$AAe?$AAm?$AA?4?$AAd?$AAl?$AAl?$AA?$AA@ 10001074     buspcie950.obj
 0001:00000090       ??_C@_1BO@DLFIJDKP@?$AA?$CF?$AAs?$AA?2?$AAS?$AAe?$AAr?$AAi?$AAa?$AAl?$AAC?$AAa?$AAb?$AAl?$AAe?$AA?$AA@ 10001090     buspcie950.obj
 0001:000000b0       ??_C@_15GANGMFKL@?$AA?$CF?$AAs?$AA?$AA@ 100010b0     buspcie950.obj
 0001:000000b8       ??_C@_11LOCGONAA@?$AA?$AA@ 100010b8     buspcie950.obj
 0001:000000bc       ??_C@_1CA@INOAHGHF@?$AAB?$AAu?$AAs?$AAA?$AAc?$AAc?$AAe?$AAs?$AAs?$AAH?$AAa?$AAn?$AAd?$AAl?$AAe?$AA?$AA@ 100010bc     buspcie950.obj
 0001:000000dc       ??_C@_1O@GBAEOCCH@?$AAP?$AAr?$AAe?$AAf?$AAi?$AAx?$AA?$AA@ 100010dc     buspcie950.obj
 0001:000000ec       ??_C@_1BE@GPBAGNPC@?$AAI?$AAs?$AAr?$AAH?$AAa?$AAn?$AAd?$AAl?$AAe?$AA?$AA@ 100010ec     buspcie950.obj
 0001:00000100       ??_C@_1BC@MCDIKBIL@?$AAI?$AAs?$AAt?$AAE?$AAv?$AAe?$AAn?$AAt?$AA?$AA@ 10001100     buspcie950.obj
 0001:00000114       ??_C@_1BG@LJAMCNJN@?$AAP?$AAo?$AAr?$AAt?$AAN?$AAu?$AAm?$AAb?$AAe?$AAr?$AA?$AA@ 10001114     buspcie950.obj
 0001:0000012c       ??_C@_1CC@KMPFMANC@?$AAD?$AAe?$AAv?$AAi?$AAc?$AAe?$AAA?$AAr?$AAr?$AAa?$AAy?$AAI?$AAn?$AAd?$AAe?$AAx?$AA?$AA@ 1000112c     buspcie950.obj
 0001:00000150       ??_C@_17DJMMGLBL@?$AAD?$AAl?$AAl?$AA?$AA@ 10001150     buspcie950.obj
 0001:00000158       ??_C@_17KKLPNNMB@?$AAC?$AAO?$AAM?$AA?$AA@ 10001158     buspcie950.obj
 0001:00000160       ??_C@_1BE@EODMIMC@?$AA?$CF?$AAs?$AA?2?$AAp?$AAo?$AAr?$AAt?$AA?$CF?$AAd?$AA?$AA@ 10001160     buspcie950.obj
 0001:00000174       ??_C@_1CM@HIMBKDJM@?$AAL?$AAi?$AAn?$AAe?$AAD?$AAr?$AAi?$AAv?$AAe?$AAr?$AAD?$AAe?$AAl?$AAa?$AAy?$AAP?$AAh?$AAa?$AAs?$AAe?$AAs?$AA?$AA@ 10001174     buspcie950.obj
 0001:000001a0       ??_C@_1CI@GLAIJPLJ@?$AAL?$AAi?$AAn?$AAe?$AAD?$AAr?$AAi?$AAv?$AAe?$AAr?$AAD?$AAe?$AAl?$AAa?$AAy?$AAB?$AAi?$AAt?$AAs?$AA?$AA@ 100011a0     buspcie950.obj
 0001:000001c8       ??_C@_1CI@OJPKJBA@?$AAB?$AAa?$AAu?$AAd?$AAr?$AAa?$AAt?$AAe?$AAM?$AAa?$AAp?$AAL?$AAi?$AAs?$AAt?$AAF?$AAr?$AAo?$AAm?$AA?$AA@ 100011c8     buspcie950.obj
 0001:000001f0       ??_C@_1CE@BHEKDMEI@?$AAB?$AAa?$AAu?$AAd?$AAr?$AAa?$AAt?$AAe?$AAM?$AAa?$AAp?$AAL?$AAi?$AAs?$AAt?$AAT?$AAo?$AA?$AA@ 100011f0     buspcie950.obj
 0001:00000214       ??_C@_1BE@DDEHHBPD@?$AAD?$AAe?$AAv?$AAC?$AAo?$AAn?$AAf?$AAi?$AAg?$AA?$AA@ 10001214     buspcie950.obj
 0001:00000228       ??_C@_17KNDIACFJ@?$AAT?$AAs?$AAp?$AA?$AA@ 10001228     buspcie950.obj
 0001:00000230       ??_C@_1BG@JDAFHBOG@?$AAI?$AAS?$AAR?$AAH?$AAa?$AAn?$AAd?$AAl?$AAe?$AAr?$AA?$AA@ 10001230     buspcie950.obj
 0001:00000248       ??_C@_1BG@NELPJJNN@?$AAI?$AAs?$AAr?$AAH?$AAa?$AAn?$AAd?$AAl?$AAe?$AAr?$AA?$AA@ 10001248     buspcie950.obj
 0001:00000260       ??_C@_1BO@KACPNJCM@?$AAi?$AAs?$AAr?$AAp?$AAc?$AAi?$AAe?$AA9?$AA5?$AA0?$AA?4?$AAd?$AAl?$AAl?$AA?$AA@ 10001260     buspcie950.obj
 0001:00000280       ??_C@_1O@MDNCMDKF@?$AAI?$AAs?$AAr?$AAD?$AAl?$AAl?$AA?$AA@ 10001280     buspcie950.obj
 0001:00000290       ??_C@_1BO@NHAHMBJD@?$AAc?$AAo?$AAm?$AAp?$AAc?$AAi?$AAe?$AA9?$AA5?$AA0?$AA?4?$AAd?$AAl?$AAl?$AA?$AA@ 10001290     buspcie950.obj
 0001:000002b0       ??_C@_1BA@CEFELOID@?$AAU?$AAa?$AAr?$AAt?$AAD?$AAl?$AAl?$AA?$AA@ 100012b0     buspcie950.obj
 0001:000002c0       ??_C@_1BA@BDHDGOBO@?$AAS?$AAy?$AAs?$AAI?$AAn?$AAt?$AAr?$AA?$AA@ 100012c0     buspcie950.obj
 0001:000002d0       ??_C@_17DJGGJCGD@?$AAI?$AAr?$AAq?$AA?$AA@ 100012d0     buspcie950.obj
 0001:000002d8       ??_C@_1BM@MHMIAMLB@?$AAI?$AAn?$AAt?$AAe?$AAr?$AAf?$AAa?$AAc?$AAe?$AAT?$AAy?$AAp?$AAe?$AA?$AA@ 100012d8     buspcie950.obj
 0001:000002f4       ??_C@_1BE@MNDDMKMB@?$AAB?$AAu?$AAs?$AAN?$AAu?$AAm?$AAb?$AAe?$AAr?$AA?$AA@ 100012f4     buspcie950.obj
 0001:00000308       ??_C@_1O@LBBNFMDB@?$AAM?$AAe?$AAm?$AAL?$AAe?$AAn?$AA?$AA@ 10001308     buspcie950.obj
 0001:00000318       ??_C@_1BA@INLDIDEN@?$AAM?$AAe?$AAm?$AAB?$AAa?$AAs?$AAe?$AA?$AA@ 10001318     buspcie950.obj
 0001:00000328       ??_C@_1M@PEPOCCHH@?$AAI?$AAo?$AAL?$AAe?$AAn?$AA?$AA@ 10001328     buspcie950.obj
 0001:00000334       ??_C@_1O@JMCNHCBG@?$AAI?$AAo?$AAB?$AAa?$AAs?$AAe?$AA?$AA@ 10001334     buspcie950.obj
 0001:00000344       ??_C@_1CE@PJBMNJAF@?$AAL?$AAi?$AAn?$AAe?$AAD?$AAr?$AAi?$AAv?$AAe?$AAr?$AAC?$AAo?$AAn?$AAt?$AAr?$AAo?$AAl?$AA?$AA@ 10001344     buspcie950.obj
 0001:00000368       ??_C@_1CE@HLGCKFJ@?$AAF?$AAl?$AAo?$AAw?$AAC?$AAt?$AAr?$AAl?$AAH?$AAi?$AAg?$AAh?$AAL?$AAe?$AAv?$AAe?$AAl?$AA?$AA@ 10001368     buspcie950.obj
 0001:0000038c       ??_C@_1CC@ELLFOF@?$AAF?$AAl?$AAo?$AAw?$AAC?$AAt?$AAr?$AAl?$AAL?$AAo?$AAw?$AAL?$AAe?$AAv?$AAe?$AAl?$AA?$AA@ 1000138c     buspcie950.obj
 0001:000003b0       ??_C@_1BO@MCGADMLE@?$AAR?$AAx?$AAI?$AAn?$AAt?$AAT?$AAr?$AAi?$AAg?$AAL?$AAe?$AAv?$AAe?$AAl?$AA?$AA@ 100013b0     buspcie950.obj
 0001:000003d0       ??_C@_1BO@ELCCHGIE@?$AAT?$AAx?$AAI?$AAn?$AAt?$AAT?$AAr?$AAi?$AAg?$AAL?$AAe?$AAv?$AAe?$AAl?$AA?$AA@ 100013d0     buspcie950.obj
 0001:000003f0       ??_C@_1CC@EKOCNIBB@?$AAC?$AAr?$AAy?$AAs?$AAt?$AAa?$AAl?$AAF?$AAr?$AAe?$AAq?$AAu?$AAe?$AAn?$AAc?$AAy?$AA?$AA@ 100013f0     buspcie950.obj
 0001:00000414       ??_C@_1BK@KAMHHDIE@?$AAB?$AAr?$AAa?$AAn?$AAd?$AAi?$AAn?$AAg?$AAF?$AAi?$AAl?$AAe?$AA?$AA@ 10001414     buspcie950.obj
 0001:00000430       ??_C@_1BM@CMGCPMHF@?$AAR?$AAe?$AAa?$AAd?$AAB?$AAr?$AAa?$AAn?$AAd?$AAF?$AAi?$AAl?$AAe?$AA?$AA@ 10001430     buspcie950.obj
 0001:0000044c       ??_C@_17KACEIPNC@?$AAK?$AAe?$AAy?$AA?$AA@ 1000144c     buspcie950.obj
 0001:00000454       ??_C@_1DC@JFNGNCBP@?$AAS?$AAe?$AAr?$AAi?$AAa?$AAl?$AA?5?$AAC?$AAa?$AAb?$AAl?$AAe?$AA?5?$AAo?$AAn?$AA?5?$AAC?$AAO?$AAM?$AA?5?$AAP?$AAo?$AAr?$AAt?$AA?$AA@ 10001454     buspcie950.obj
 0001:00000488       ??_C@_1DK@IPGGKJ@?$AAH?$AAa?$AAy?$AAe?$AAs?$AA?5?$AAC?$AAo?$AAm?$AAp?$AAa?$AAt?$AAi?$AAb?$AAl?$AAe?$AA?5?$AAo?$AAn?$AA?5?$AAC?$AAO?$AAM?$AA?5?$AAP?$AAo?$AAr?$AAt?$AA?$AA@ 10001488     buspcie950.obj
 0001:000004c4       ??_C@_1M@FFLAJJMG@?$AA?$DM?$AAE?$AAN?$AAD?$AA?$DO?$AA?$AA@ 100014c4     ConfigParser.obj
 0001:000004d0       ??_C@_1CG@LGKPGFHM@?$AAN?$AAo?$AA?5?$AAC?$AAo?$AAn?$AAt?$AAr?$AAo?$AAl?$AA?5?$AA?$CI?$AAR?$AAS?$AA2?$AA3?$AA2?$AA?$CJ?$AA?$AA@ 100014d0     ConfigParser.obj
 0001:000004f8       ??_C@_1CO@KJKNEDLA@?$AAL?$AAo?$AAw?$AA?5?$AAE?$AAn?$AAa?$AAb?$AAl?$AAe?$AA?5?$AA?$CI?$AAR?$AAS?$AA4?$AA2?$AA2?$AA?1?$AA4?$AA8?$AA5?$AA?$CJ?$AA?$AA@ 100014f8     ConfigParser.obj
 0001:00000528       ??_C@_1BI@LGOMGNKN@?$AAH?$AAi?$AAg?$AAh?$AA?5?$AAE?$AAn?$AAa?$AAb?$AAl?$AAe?$AA?$AA@ 10001528     ConfigParser.obj
 0001:00000540       ??_C@_19BIEPDBPA@?$AAT?$AAy?$AAp?$AAe?$AA?$AA@ 10001540     ConfigParser.obj
 0001:0000054c       ??_C@_1CI@IMABDCBP@?$AAL?$AAi?$AAn?$AAe?$AA_?$AAD?$AAr?$AAi?$AAv?$AAe?$AAr?$AA_?$AAC?$AAo?$AAn?$AAt?$AAr?$AAo?$AAl?$AA?$AA@ 1000154c     ConfigParser.obj
 0001:00000574       ??_C@_1BK@CENGCIFF@?$AAT?$AAo?$AA_?$AAB?$AAa?$AAu?$AAd?$AA_?$AAR?$AAa?$AAt?$AAe?$AA?$AA@ 10001574     ConfigParser.obj
 0001:00000590       ??_C@_1BO@CILDMCD@?$AAF?$AAr?$AAo?$AAm?$AA_?$AAB?$AAa?$AAu?$AAd?$AA_?$AAR?$AAa?$AAt?$AAe?$AA?$AA@ 10001590     ConfigParser.obj
 0001:000005b0       ??_C@_1CC@FHAFLLA@?$AAB?$AAa?$AAu?$AAd?$AAr?$AAa?$AAt?$AAe?$AA_?$AAM?$AAa?$AAp?$AAp?$AAi?$AAn?$AAg?$AA?$AA@ 100015b0     ConfigParser.obj
 0001:000005d4       ??_C@_1BE@GELDBLFK@?$AAT?$AAa?$AAb?$AA_?$AAA?$AAb?$AAo?$AAu?$AAt?$AA?$AA@ 100015d4     ConfigParser.obj
 0001:000005e8       ??_C@_1DA@NCKAKAMN@?$AAT?$AAa?$AAb?$AA_?$AAL?$AAi?$AAn?$AAe?$AA_?$AAD?$AAr?$AAi?$AAv?$AAe?$AAr?$AA_?$AAC?$AAo?$AAn?$AAt?$AAr?$AAo?$AAl?$AA?$AA@ 100015e8     ConfigParser.obj
 0001:00000618       ??_C@_1CA@LJNFGPHD@?$AAT?$AAa?$AAb?$AA_?$AAF?$AAi?$AAf?$AAo?$AA_?$AAL?$AAe?$AAv?$AAe?$AAl?$AAs?$AA?$AA@ 10001618     ConfigParser.obj
 0001:00000638       ??_C@_1CK@NLOLPFMM@?$AAT?$AAa?$AAb?$AA_?$AAB?$AAa?$AAu?$AAd?$AAr?$AAa?$AAt?$AAe?$AA_?$AAM?$AAa?$AAp?$AAp?$AAi?$AAn?$AAg?$AA?$AA@ 10001638     ConfigParser.obj
 0001:00000664       ??_C@_1CM@OFMOCLCD@?$AAT?$AAa?$AAb?$AA_?$AAC?$AAr?$AAy?$AAs?$AAt?$AAa?$AAl?$AA_?$AAF?$AAr?$AAe?$AAq?$AAu?$AAe?$AAn?$AAc?$AAy?$AA?$AA@ 10001664     ConfigParser.obj
 0001:00000690       ??_C@_1BI@LMBHJBLG@?$AAT?$AAa?$AAb?$AA_?$AAO?$AAp?$AAt?$AAi?$AAo?$AAn?$AAs?$AA?$AA@ 10001690     ConfigParser.obj
 0001:000006a8       ??_C@_1DG@MMINKBLM@?$AAF?$AAl?$AAo?$AAw?$AA_?$AAC?$AAo?$AAn?$AAt?$AAr?$AAo?$AAl?$AA_?$AAO?$AAf?$AAf?$AA_?$AAL?$AAe?$AAv?$AAe?$AAl?$AA_?$AAM?$AAa?$AAx?$AA?$AA@ 100016a8     ConfigParser.obj
 0001:000006e0       ??_C@_1DG@FFKMCLJC@?$AAF?$AAl?$AAo?$AAw?$AA_?$AAC?$AAo?$AAn?$AAt?$AAr?$AAo?$AAl?$AA_?$AAO?$AAf?$AAf?$AA_?$AAL?$AAe?$AAv?$AAe?$AAl?$AA_?$AAM?$AAi?$AAn?$AA?$AA@ 100016e0     ConfigParser.obj
 0001:00000718       ??_C@_1DE@JAENBBJL@?$AAF?$AAl?$AAo?$AAw?$AA_?$AAC?$AAo?$AAn?$AAt?$AAr?$AAo?$AAl?$AA_?$AAO?$AAn?$AA_?$AAL?$AAe?$AAv?$AAe?$AAl?$AA_?$AAM?$AAa?$AAx?$AA?$AA@ 10001718     ConfigParser.obj
 0001:0000074c       ??_C@_1DE@JGMJLLF@?$AAF?$AAl?$AAo?$AAw?$AA_?$AAC?$AAo?$AAn?$AAt?$AAr?$AAo?$AAl?$AA_?$AAO?$AAn?$AA_?$AAL?$AAe?$AAv?$AAe?$AAl?$AA_?$AAM?$AAi?$AAn?$AA?$AA@ 1000174c     ConfigParser.obj
 0001:00000780       ??_C@_1DO@FFHHIFI@?$AAR?$AAx?$AA_?$AAI?$AAn?$AAt?$AAe?$AAr?$AAr?$AAu?$AAp?$AAt?$AA_?$AAT?$AAr?$AAi?$AAg?$AAg?$AAe?$AAr?$AA_?$AAL?$AAe?$AAv?$AAe?$AAl?$AA_?$AAM?$AAa?$AAx?$AA?$AA@ 10001780     ConfigParser.obj
 0001:000007c0       ??_C@_1DO@JMHGPCHG@?$AAR?$AAx?$AA_?$AAI?$AAn?$AAt?$AAe?$AAr?$AAr?$AAu?$AAp?$AAt?$AA_?$AAT?$AAr?$AAi?$AAg?$AAg?$AAe?$AAr?$AA_?$AAL?$AAe?$AAv?$AAe?$AAl?$AA_?$AAM?$AAi?$AAn?$AA?$AA@ 100017c0     ConfigParser.obj
 0001:00000800       ??_C@_1DO@HONDFPK@?$AAT?$AAx?$AA_?$AAI?$AAn?$AAt?$AAe?$AAr?$AAr?$AAu?$AAp?$AAt?$AA_?$AAT?$AAr?$AAi?$AAg?$AAg?$AAe?$AAr?$AA_?$AAL?$AAe?$AAv?$AAe?$AAl?$AA_?$AAM?$AAa?$AAx?$AA?$AA@ 10001800     ConfigParser.obj
 0001:00000840       ??_C@_1DO@JOMMLPNE@?$AAT?$AAx?$AA_?$AAI?$AAn?$AAt?$AAe?$AAr?$AAr?$AAu?$AAp?$AAt?$AA_?$AAT?$AAr?$AAi?$AAg?$AAg?$AAe?$AAr?$AA_?$AAL?$AAe?$AAv?$AAe?$AAl?$AA_?$AAM?$AAi?$AAn?$AA?$AA@ 10001840     ConfigParser.obj
 0001:00000880       ??_C@_1BO@CLLBHNOO@?$AAF?$AAl?$AAo?$AAw?$AA_?$AAO?$AAf?$AAf?$AA_?$AAL?$AAe?$AAv?$AAe?$AAl?$AA?$AA@ 10001880     ConfigParser.obj
 0001:000008a0       ??_C@_1BM@FKEALHLG@?$AAF?$AAl?$AAo?$AAw?$AA_?$AAO?$AAn?$AA_?$AAL?$AAe?$AAv?$AAe?$AAl?$AA?$AA@ 100018a0     ConfigParser.obj
 0001:000008c0       ??_C@_1EA@FCDBIJCN@?$AAR?$AAe?$AAc?$AAe?$AAi?$AAv?$AAe?$AA_?$AAI?$AAn?$AAt?$AAe?$AAr?$AAr?$AAu?$AAp?$AAt?$AA_?$AAT?$AAr?$AAi?$AAg?$AAg?$AAe?$AAr?$AA_?$AAL?$AAe?$AAv?$AAe?$AAl?$AA?$AA@ 100018c0     ConfigParser.obj
 0001:00000900       ??_C@_1EC@JOHHNGND@?$AAT?$AAr?$AAa?$AAn?$AAs?$AAm?$AAi?$AAt?$AA_?$AAI?$AAn?$AAt?$AAe?$AAr?$AAr?$AAu?$AAp?$AAt?$AA_?$AAT?$AAr?$AAi?$AAg?$AAg?$AAe?$AAr?$AA_?$AAL?$AAe?$AAv?$AAe?$AAl@ 10001900     ConfigParser.obj
 0001:00000944       ??_C@_1BI@GEBICGMH@?$AAF?$AAi?$AAf?$AAo?$AA_?$AAL?$AAe?$AAv?$AAe?$AAl?$AAs?$AA?$AA@ 10001944     ConfigParser.obj
 0001:0000095c       ??_C@_1CE@FHCKENKN@?$AAC?$AAr?$AAy?$AAs?$AAt?$AAa?$AAl?$AA_?$AAF?$AAr?$AAe?$AAq?$AAu?$AAe?$AAn?$AAc?$AAy?$AA?$AA@ 1000195c     ConfigParser.obj
 0001:00000980       ??_C@_1M@MNHBCACD@?$AAT?$AAi?$AAt?$AAl?$AAe?$AA?$AA@ 10001980     ConfigParser.obj
 0001:0000098c       ??_C@_1CE@EOJPOKCA@?$AAA?$AAp?$AAp?$AAl?$AAi?$AAc?$AAa?$AAt?$AAi?$AAo?$AAn?$AA_?$AAT?$AAi?$AAt?$AAl?$AAe?$AA?$AA@ 1000198c     ConfigParser.obj
 0001:000009b0       ??_C@_1BI@MHELFDAB@?$AA?2?$AAW?$AAi?$AAn?$AAd?$AAo?$AAw?$AAs?$AA?2?$AA?$CF?$AAs?$AA?$AA@ 100019b0     ConfigParser.obj
 0001:000009c8       ??_C@_15JJPIMNBO@?$AAr?$AAb?$AA?$AA@ 100019c8     ConfigParser.obj
 0001:000009f8       ?DllEntry@@YAHPAUHINSTANCE__@@KPAX@Z 100019f8 f   buspcie950.obj
 0001:00000a94       ?Deinit@@YAXPAX@Z          10001a94 f   buspcie950.obj
 0001:00000d80       ?Init@@YAPAXPBG@Z          10001d80 f   buspcie950.obj
 0001:00002004       _tfsubstring               10003004 f   ConfigParser.obj
 0001:00002054       ?_ffeosubsec@@YAHPAXQAG@Z  10003054 f   ConfigParser.obj
 0001:000020a0       ?ValidateCrystalFrequency@@YAHH@Z 100030a0 f   ConfigParser.obj
 0001:000021c8       ?ValidateValues@@YAXPAU_CONFIG_DATA_@@@Z 100031c8 f   ConfigParser.obj
 0001:00002300       ?_textractValue@@YAPAGPAG@Z 10003300 f   ConfigParser.obj
 0001:00002348       ParseConfigFile            10003348 f   ConfigParser.obj
 0001:00002a9c       BusTransBusAddrToStatic    10003a9c f   ceddk:CEDDK.dll
 0001:00002aac       BusTransBusAddrToVirtual   10003aac f   ceddk:CEDDK.dll
 0001:00002abc       CreateBusAccessHandle      10003abc f   ceddk:CEDDK.dll
 0001:00002acc       EventModify                10003acc f   coredll:COREDLL.dll
 0001:00002adc       KernelLibIoControl         10003adc f   coredll:COREDLL.dll
 0001:00002aec       DisableThreadLibraryCalls  10003aec f   coredll:COREDLL.dll
 0001:00002afc       InterruptDone              10003afc f   coredll:COREDLL.dll
 0001:00002b0c       InterlockedExchange        10003b0c f   coredll:COREDLL.dll
 0001:00002b1c       WaitForSingleObject        10003b1c f   coredll:COREDLL.dll
 0001:00002b2c       CloseHandle                10003b2c f   coredll:COREDLL.dll
 0001:00002b3c       DeactivateDevice           10003b3c f   coredll:COREDLL.dll
 0001:00002b4c       RegQueryValueExW           10003b4c f   coredll:COREDLL.dll
 0001:00002b5c       RegSetValueExW             10003b5c f   coredll:COREDLL.dll
 0001:00002b6c       GetDeviceInformationByDeviceHandle 10003b6c f   coredll:COREDLL.dll
 0001:00002b7c       ActivateDeviceEx           10003b7c f   coredll:COREDLL.dll
 0001:00002b8c       RegCreateKeyExW            10003b8c f   coredll:COREDLL.dll
 0001:00002b9c       wsprintfW                  10003b9c f   coredll:COREDLL.dll
 0001:00002bac       CreateThread               10003bac f   coredll:COREDLL.dll
 0001:00002bbc       InterruptInitialize        10003bbc f   coredll:COREDLL.dll
 0001:00002bcc       CreateEventW               10003bcc f   coredll:COREDLL.dll
 0001:00002bdc       LoadIntChainHandler        10003bdc f   coredll:COREDLL.dll
 0001:00002bec       RegCloseKey                10003bec f   coredll:COREDLL.dll
 0001:00002bfc       RegOpenKeyExW              10003bfc f   coredll:COREDLL.dll
 0001:00002c0c       __GSHandlerCheckCommon     10003c0c f   corelib0:gshandler.obj
 0001:00002c48       __GSHandlerCheck           10003c48 f   corelib0:gshandler.obj
 0001:00002c6c       __security_check_cookie    10003c6c f   corelib0:armsecgs.obj
 0001:00002c80       __gsfailure                10003c80 f   corelib0:armsecgs.obj
 0001:00002cc4       wcstoul                    10003cc4 f   corelib1:COREDLL.dll
 0001:00002cd4       wcslen                     10003cd4 f   corelib1:COREDLL.dll
 0001:00002ce4       free                       10003ce4 f   corelib1:COREDLL.dll
 0001:00002cf4       malloc                     10003cf4 f   corelib1:COREDLL.dll
 0001:00002d04       wcstol                     10003d04 f   corelib1:COREDLL.dll
 0001:00002d14       wcscpy                     10003d14 f   corelib1:COREDLL.dll
 0001:00002d24       memcpy                     10003d24 f   corelib1:COREDLL.dll
 0001:00002d34       wcschr                     10003d34 f   corelib1:COREDLL.dll
 0001:00002d44       wcsrchr                    10003d44 f   corelib1:COREDLL.dll
 0001:00002d54       fgetws                     10003d54 f   corelib1:COREDLL.dll
 0001:00002d64       wcscmp                     10003d64 f   corelib1:COREDLL.dll
 0001:00002d74       fclose                     10003d74 f   corelib1:COREDLL.dll
 0001:00002d84       _wtol                      10003d84 f   corelib1:COREDLL.dll
 0001:00002d94       feof                       10003d94 f   corelib1:COREDLL.dll
 0001:00002da4       _wfopen                    10003da4 f   corelib1:COREDLL.dll
 0001:00002db4       swprintf                   10003db4 f   corelib1:COREDLL.dll
 0001:00002dc4       __report_gsfailure         10003dc4 f   corelib1:COREDLL.dll
 0001:00002de0       __IMPORT_DESCRIPTOR_CEDDK  10003de0     ceddk:CEDDK.dll
 0001:00002df4       __IMPORT_DESCRIPTOR_COREDLL 10003df4     coredll:COREDLL.dll
 0001:00002e08       __NULL_IMPORT_DESCRIPTOR   10003e08     ceddk:CEDDK.dll
 0002:00000000       __imp_BusTransBusAddrToVirtual 10004000     ceddk:CEDDK.dll
 0002:00000004       __imp_CreateBusAccessHandle 10004004     ceddk:CEDDK.dll
 0002:00000008       __imp_BusTransBusAddrToStatic 10004008     ceddk:CEDDK.dll
 0002:0000000c       \177CEDDK_NULL_THUNK_DATA  1000400c     ceddk:CEDDK.dll
 0002:00000010       __imp_EventModify          10004010     coredll:COREDLL.dll
 0002:00000014       __imp_KernelLibIoControl   10004014     coredll:COREDLL.dll
 0002:00000018       __imp_DisableThreadLibraryCalls 10004018     coredll:COREDLL.dll
 0002:0000001c       __imp_InterruptDone        1000401c     coredll:COREDLL.dll
 0002:00000020       __imp_InterlockedExchange  10004020     coredll:COREDLL.dll
 0002:00000024       __imp_WaitForSingleObject  10004024     coredll:COREDLL.dll
 0002:00000028       __imp_CloseHandle          10004028     coredll:COREDLL.dll
 0002:0000002c       __imp_DeactivateDevice     1000402c     coredll:COREDLL.dll
 0002:00000030       __imp_RegQueryValueExW     10004030     coredll:COREDLL.dll
 0002:00000034       __imp_RegSetValueExW       10004034     coredll:COREDLL.dll
 0002:00000038       __imp_GetDeviceInformationByDeviceHandle 10004038     coredll:COREDLL.dll
 0002:0000003c       __imp_ActivateDeviceEx     1000403c     coredll:COREDLL.dll
 0002:00000040       __imp_RegCreateKeyExW      10004040     coredll:COREDLL.dll
 0002:00000044       __imp_wsprintfW            10004044     coredll:COREDLL.dll
 0002:00000048       __imp_CreateThread         10004048     coredll:COREDLL.dll
 0002:0000004c       __imp_InterruptInitialize  1000404c     coredll:COREDLL.dll
 0002:00000050       __imp_CreateEventW         10004050     coredll:COREDLL.dll
 0002:00000054       __imp_LoadIntChainHandler  10004054     coredll:COREDLL.dll
 0002:00000058       __imp_RegCloseKey          10004058     coredll:COREDLL.dll
 0002:0000005c       __imp_RegOpenKeyExW        1000405c     coredll:COREDLL.dll
 0002:00000060       __imp_wcstoul              10004060     corelib1:COREDLL.dll
 0002:00000064       __imp_wcslen               10004064     corelib1:COREDLL.dll
 0002:00000068       __imp_free                 10004068     corelib1:COREDLL.dll
 0002:0000006c       __imp_malloc               1000406c     corelib1:COREDLL.dll
 0002:00000070       __imp_wcstol               10004070     corelib1:COREDLL.dll
 0002:00000074       __imp_wcscpy               10004074     corelib1:COREDLL.dll
 0002:00000078       __imp_memcpy               10004078     corelib1:COREDLL.dll
 0002:0000007c       __imp_wcschr               1000407c     corelib1:COREDLL.dll
 0002:00000080       __imp_wcsrchr              10004080     corelib1:COREDLL.dll
 0002:00000084       __imp_fgetws               10004084     corelib1:COREDLL.dll
 0002:00000088       __imp_wcscmp               10004088     corelib1:COREDLL.dll
 0002:0000008c       __imp_fclose               1000408c     corelib1:COREDLL.dll
 0002:00000090       __imp__wtol                10004090     corelib1:COREDLL.dll
 0002:00000094       __imp_feof                 10004094     corelib1:COREDLL.dll
 0002:00000098       __imp__wfopen              10004098     corelib1:COREDLL.dll
 0002:0000009c       __imp_swprintf             1000409c     corelib1:COREDLL.dll
 0002:000000a0       __imp___report_gsfailure   100040a0     corelib1:COREDLL.dll
 0002:000000a4       \177COREDLL_NULL_THUNK_DATA 100040a4     coredll:COREDLL.dll
 0002:000000a8       ?dpCurSettings@@3U_DBGPARAM@@A 100040a8     buspcie950.obj
 0002:000004ec       __security_cookie          100044ec     corelib0:seccinit.obj
 0002:000004f0       __security_cookie_complement 100044f0     corelib0:seccinit.obj
 0002:000004f8       ?Pcie950BusInfo@@3UPCIE950_BUS_INFO@@A 100044f8     buspcie950.obj
 0002:00000598       ?m_pDispatchThread@@3PAXA  10004598     buspcie950.obj

 entry point at        0000:00000000

 Static symbols

 0001:00000a10       ?BusIstThread@@YAKPAX@Z    10001a10 f   buspcie950.obj
 0001:00000b60       ?ReadKeyList@@YAHPAUHKEY__@@PBGKPAK2@Z 10001b60 f   buspcie950.obj
 0001:00000c80       ?ReadKeyDword@@YAHPAUHKEY__@@PBGPAK@Z 10001c80 f   buspcie950.obj
 0001:00000cdc       ?WriteKeyDword@@YAHPAUHKEY__@@PBGK@Z 10001cdc f   buspcie950.obj
 0001:00000d20       ?WriteKeyString@@YAHPAUHKEY__@@PBG1@Z 10001d20 f   buspcie950.obj
